:04000000883100281B
:1000080070082000A0008031141D1A283000161D29
:100018001928161112082000EA00300013082000E1
:10002800EB000130E6000030E7003C282000901E7D
:100038003C28A030680786000030693D870023000F
:1000480019088100A0302000680784000030693D4D
:1000580085000008233A031D3928FF30E800FF30E7
:10006800E9000130DF000030E000E80A0319E90A7E
:060078002008F000090061
:0E007E0055303C008F00AA308F000F14080090
:0E008C0055303C008F00AA308F000F10080086
:10009A0022003D08053C031857280C303D0203187E
:1000AA0057285C283D08173C031C5C285E28F00191
:1000BA00102B3E08003A031D06294008031966283A
:1000CA004620BC2822003F083D009000012922005A
:1000DA003F083D009100012922003F083D0092009F
:1000EA00012922003F083D009400012922003F080F
:1000FA003D009500012922003F083D009C0001298E
:10010A0022003F083D009D00012922003F083D00D2
:10011A009E00012922003F083D009F00012922007C
:10012A003F083D00A000012922003F083D00A10030
:10013A00012922003F083D00A200012922003F08B0
:10014A003D00A300012922003F083D00A400012927
:10015A0022003F083D00A500012922003F083D007A
:10016A00A600012922003F083D00A700012922001C
:10017A003D08003A031967283D08013A03196C281B
:10018A003D08023A031971283D08043A03197628F2
:10019A003D08053A03197B283D080C3A03198028C3
:1001AA003D080D3A031985283D080E3A03198A2895
:1001BA003D080F3A03198F283D08103A031994286D
:1001CA003D08113A031999283D08123A03199E2845
:1001DA003D08133A0319A3283D08143A0319A8281D
:1001EA003D08153A0319AD283D08163A0319B228F5
:1001FA003D08173A0319B7282200400803190629AF
:10020A003F2022003E08013A031D2F2A4008031905
:10021A000F29462022003D08C100AD2941083C00B3
:10022A0090002A2A220041083C0091002A2A220032
:10023A0041083C0092002A2A220041083C0093000F
:10024A002A2A220041083C0098002A2A2200410852
:10025A003C0099002A2A220041083C009A002A2AD6
:10026A00220041083C009B002A2A220041083C0047
:10027A009C002A2A220041083C009D002A2A2200CA
:10028A0041083C009E002A2A220041083C009400B2
:10029A002A2A220041083C0095002A2A2200410805
:1002AA003C0097002A2A220041083C00A0002A2A82
:1002BA00220041083C00A1002A2A220041083C00F1
:1002CA00A2002A2A220041083C00A4002A2A22006D
:1002DA0041083C00A5002A2A220041083C00A80047
:1002EA002A2A220041083C00A9002A2A22004108A1
:1002FA003C00AA002A2A220041083C00AB002A2A14
:10030A00220041083C00A7002A2A220041083C009A
:10031A00A6002A2A220041083C00AD002A2A22000F
:10032A0041083C00AC002A2A220041083C00960001
:10033A002A2A220041083C009F002A2A220041085A
:10034A003C00A3002A2A220041083C00AE002A2AC7
:10035A0022003F08003A031913293F08013A0319FA
:10036A0017293F08023A03191C293F08033A0319BF
:10037A0021293F08043A031926293F08053A031997
:10038A002B293F08063A031930293F08073A03196F
:10039A0035293F08083A03193A293F08093A031947
:1003AA003F293F080A3A031944293F080B3A03191F
:1003BA0049293F080C3A03194E293F080D3A0319F7
:1003CA0053293F080E3A031958293F080F3A0319CF
:1003DA005D293F08103A031962293F08113A0319A7
:1003EA0067293F08123A03196C293F08133A03197F
:1003FA0071293F08143A031976293F08153A031957
:10040A007B293F08163A031980293F08173A03192E
:10041A0085293F08183A03198A293F08193A031906
:10042A008F293F081A3A031994293F081B3A0319DE
:10043A0099293F081C3A03199E293F081D3A0319B6
:10044A00A3293F081E3A0319A829220040080319C4
:10045A002F2A3F20C92A22003E18362A21000C10D2
:10046A00382A21000C140E2B22003E183F2A2100A4
:10047A008C10412A21008C140E2B22003E18482A87
:10048A0021000C114A2A21000C150E2B22003E18BD
:10049A00512A21000C12532A21000C160E2B22007D
:1004AA003E185A2A21008C125C2A21008C160E2B27
:1004BA0022003E18632A21000D12652A21000D161A
:1004CA000E2B22003E186C2A21008D126E2A210062
:1004DA008D160E2B22003E18752A21000D13772A3D
:1004EA0021000D170E2B22003E187E2A21008D13A3
:1004FA00802A21008D170E2B22003E18872A210000
:10050A000E10892A21000E140E2B22003E18902A62
:10051A0021008E10922A21008E140E2B22003E18E2
:10052A00992A21000E119B2A21000E150E2B22005A
:10053A003E18A22A21008E11A42A21008E150E2B04
:10054A0022003E18AB2A21000E12AD2A21000E16F7
:10055A000E2B22003E18B42A21008E12B62A210040
:10056A008E160E2B22003E18BD2A21000E13BF2A1A
:10057A0021000E170E2B22003E18C62A21008E13C8
:10058A00C82A21008E170E2B22003D08003A0319B3
:10059A00302A3D08013A0319392A3D08023A03195B
:1005AA00422A3D08043A03194B2A3D08053A031921
:1005BA00542A3D080C3A03195D2A3D080D3A0319DD
:1005CA00662A3D080E3A03196F2A3D080F3A0319A5
:1005DA00782A3D08103A0319812A3D08113A03196D
:1005EA008A2A3D08123A0319932A3D08133A031935
:1005FA009C2A3D08143A0319A52A3D08153A0319FD
:10060A00AE2A3D08163A0319B72A3D08173A0319C4
:08061A00C02AFF30F0000800C7
:1006220022003A08BD003B08BE003C08BF00013072
:06063200C0004D2008008D
:1006380022002A082100C40022002B082100C5003E
:1006480022002C082100C60022002D082100C70026
:1006580022002E082100C00022002F082100C1001E
:10066800220030082100C200220031082100C30006
:10067800220032082100CC00220033082100CD00DE
:10068800220034082100CE00220035082100CF00C6
:10069800220036082100C800220037082100C900BE
:1006A800220038082100CA00220039082100CB00A6
:0206B800080038
:1006BA0021006F08393C031C692B30306F02031C80
:0C06CA00692B0130F0006A2BF0010800E1
:1006D60018302200BA00BB011430BC0011231930B7
:1006E6002200BA000130BB000A30BC00112308000A
:1006F60023009E1690309D002000901E862B23001E
:080706001908F0007F2B080028
:10070E00F501F60180307606F00080307002031D90
:10071E00932B22002E0875020318B82B22007508A1
:10072E00F4002A08F0002B08F1002C08F2002D0826
:10073E00F30074080319A92BF336F20CF10CF00C2C
:10074E00FF3EA12B0130F0057018B02B22000E10C9
:10075E00B22B22000E148E148E10F50A0319F60A0F
:04076E00892B0800CB
:100772002100ED01EE012200A801A90121006A0871
:10078200031DD32B6408F0006508F100F201F301A8
:100792007008E6007108E700FF306205E8006308B0
:1007A200FF39E900EB01EC0100306C02031DDB2B89
:1007B20008306B0203184B2C6608670403190E2CD1
:1007C2006B08F2006608F0006708F100720803196E
:1007D200EE2BF136F00CFF3EE82B01307005F300F2
:1007E2007108F4000030F4056B08073CF0006C0857
:1007F200031C013EF101F1027008F2007308F000DF
:100802007408F100720803190A2CF035F10DFF3E4D
:10081200042C7008ED047108EE04680869040319D9
:10082200462C08306B07F00000306C3DF100700878
:10083200F2006808F0006908F10072080319252C1B
:10084200F136F00CFF3E1F2C01307005F3007108E9
:10085200F4000030F4056B08073CF0006C08031C40
:10086200013EF101F1027008F2007308F000740811
:10087200F10072080319412CF035F10DFF3E3B2CBB
:1008820070082200A8047108A9042100EB0A0319C8
:10089200EC0AD52B660867040319632C0030660541
:1008A2002200A00021006708FF392200A1002100D8
:1008B2006D082200A00421006E082200A10400306D
:1008C200A200A30021006808690403197F2CFF30ED
:1008D20068052200A400210069082200A50000305A
:1008E200A505A7012508A6002408A500A40128083B
:1008F200A4042908A5040030A600A7002100660868
:10090200670403199A2C68086904031D9A2C2200B3
:100912002008AA002108AB002208AC002308AD0081
:100922001030AE00872322000D160C110E150E1189
:10093200D92C2100680869040319B52C66086704DC
:10094200031DB52C22002408AA002508AB002608A6
:10095200AC002708AD002030AE00872322000C1522
:100962000D120E150E11D92C210068086904031905
:10097200D62C660867040319D62C22002108AD0084
:100982002008AC00AA01AB012408AA042508AB0484
:100992002608AC042708AD042030AE0087232200CD
:1009A2000D120C110E150E11D92C22000D160C155C
:0209B20008003B
:1009B400210062085A3C031CE62C41306202031CED
:0C09C400E62C0130F000E72CF0010800E8
:1009D000210062085A3C031CF22C41306202031CC5
:0A09E000F22CE2166208F000080095
:1009EA006B23FF302200AA00FF30AB000030AC00BE
:1009FA000030AD00FF30AE00FF30AF00FF30B00076
:100A0A00FF30B100FF30B200FF30B3000030B40055
:100A1A000030B500FF30B600FF30B7000030B80034
:0A0A2A000030B9001C237B230800F4
:100A340021006208663C031C262D61306202031CFF
:100A4400262D0130F000272DF0017008E300620824
:100A5400463C031C342D41306202031C342D01300A
:100A6400F000352DF0017008E3046208EF005D2307
:0A0A74006308F0047008E3000800B6
:100A7E0021006208203A03194F2D62080D3C031C19
:100A8E004D2D09306202031C4D2D4F2DF001512DBD
:060A9E000130F000080029
:100AA4002100DC01DD01E001E1015A0884005B085A
:100AB40085000008E2003F2570080319652DDA0A55
:100AC4000319DB0A572D5A0884005B0885000008C7
:100AD4002D3A031D742DDC0A0319DD0ADA0A031901
:100AE400DB0A7F2D5A0884005B08850000082B3A36
:100AF400031D7F2DDA0A0319DB0A5A08F0005B088C
:100B0400F100DA0A0319DB0A700884007108850011
:100B14000008DE00DF010030DF005E08E2001A2575
:100B240070080319BD2D5E08E200DA247008031969
:100B3400A12D5E08E200E8247008DE00DF015E08F3
:100B4400EF005D2370080319AC2D3030DE02003055
:100B5400DF3BB02D5730DE020030DF3BE035E10DE6
:100B6400E035E10DE035E10DE035E10D5E08E0072B
:100B74000030E13D7F2D5C085D040319CA2D600837
:100B8400003CF0006108031C013EF101F102CE2D8E
:0A0B94006008F0006108F10008009D
:100B9E0021005A08F4005B08F5007408F20075088D
:100BAE00F300F40A0319F50A5C08F0005D08F10081
:100BBE00DC0A0319DD0A70088400710885007208CA
:100BCE00860073088700000881007208840073088D
:100BDE00850000080319F42DD42D5A08F0005B0887
:040BEE00F10008000A
:100BF200F301F40180307406F00080307002031DAE
:100C0200052E21005C0873020318322E8030740610
:100C1200F00080307002031D102E10307302031892
:100C22002A2E21007308F2005A08F0005B08F10036
:100C320072080319202EF136F00CFF3E1A2E0130F5
:100C4200F0057018272E22000E10292E22000E14F5
:100C52002C2E22000E108E148E10F30A0319F40AA1
:0A0C6200FB2D22000E150E110800F4
:100C6C0021005A08F2005B08F3005D08F0005E08F2
:100C7C00F1000130DD020030DE3B70087104031915
:100C8C00512E72088600730887005C088100F20AF6
:100C9C000319F30A3B2E5A08F0005B08F100080018
:100CAC0021005A08F2005B08F3007208F000730888
:100CBC00F100F20A0319F30A700884007108850028
:100CCC00000803196A2E5B2E5A087202F0005B08AA
:0E0CDC00733BF1000130F0020030F13B0800E4
:100CEA002100DA01DB0180305B06F00080307002FF
:100CFA00031D812E10305A020318B62EE201E301B9
:100D0A00E401E5015A08F0000030E6008030E7000F
:100D1A0070080319942EE736E60CFF3E8E2E5A0809
:100D2A00F0000130E8000030E90070080319A12E34
:100D3A00E835E90DFF3E9B2E0130EA00B923023067
:100D4A00FB000430FC00BA30FD00FD0BAA2EFC0BA0
:100D5A00AA2EFB0BAA2E00002100DA0A0319DB0ACD
:100D6A00782EE201E301E401E501E601E701E80189
:080D7A00E901EA01B9230800B8
:100D82000F303C00960031008C018D0130008D0146
:100D9200B3308C00BA30940095019601043097006C
:0A0DA20020001411210014150800B0
:100DAC0015303C00A40012303D00A40023009F1518
:100DBC0044309B0000309C001E15F5242100901639
:100DCC000530FB000F30FC00F130FD00FD0BEC2E6C
:0A0DDC00FC0BEC2EFB0BEC2E0800C4
:100DE600F83021009900FA308C00AF308D00E830E1
:100DF6008E0022008E018C018D01103023008C00A4
:100E06008D018E0126008C018D018E0122000D17A9
:020E16000800D2
:100E180012001E00F003031D0C2FF103031D0C2FFD
:020E28000800C0
:0E0E2A0022000E108E100E110C150D16080071
:10100000CA228031F326883180311527883180311A
:10101000C12688318031D62688318B170B17523084
:10102000FB002B30FC000030FD00FD0B1528FC0BF5
:101030001528FB0B1528000080317526883180317A
:101040007526883101302000EE000030EF002000CE
:101050005F08600403193029DF01E00141302100FD
:10106000DA000030DB00A030DC000030DD00803131
:10107000CF25883120004708393A031D9D284808AC
:10108000353A031D9D282100BE01BF0100303F02FB
:10109000031D4C2804303E0203187A2861303E07B5
:1010A000860000303F3D870009303E07F0000030E9
:1010B0003F3DF1004130700784000030713D8500F4
:1010C0000008810032303E07860000303F3D870037
:1010D0000D303E07F00000303F3DF1004130700719
:1010E00084000030713D850000088100BE0A0319AC
:1010F000BF0A46283230DA000030DB00803152254A
:1011000088317008D8007108D9006130DA000030E9
:10111000DB008031522588317008E6007108E70055
:10112000E201E301E401E5010130EA005808E800CA
:101130005908E9008031B923883120004708393A3D
:10114000031D0A294808323A031D0A2980317526F1
:1011500088312000B001B10121302100DA000030D7
:10116000DB00DC010F30DD000030DE008031362690
:101170008831BE01BF013E08F0003F08F100F035A4
:10118000F10D0930F0070030F13D41307007840067
:101190000030713D85000008233A03190A293E08F2
:1011A000F2003F08F300F235F30D09307207F0004A
:1011B0000030733DF1004130700784000030713D14
:1011C000850000082000BE000A307207F0000030E1
:1011D000733DF1004130700784000030713D85009F
:1011E0000008BF00213021003E07D80000303F3DFD
:1011F000D9003E30DA000030DB00803152258831E2
:10120000580886005908870070088100BE0A031933
:10121000BF0ABB2820004708393A031D3029480877
:10122000383A031D30294A08B9004B08BA00393052
:101230002100DA000030DB00803152258831003097
:101240007106031D252930307006031D2B2920004F
:10125000B701B801302920000130B7000030B800D4
:101260008D1E36290130EC000030ED008D1A3D292D
:101270006C086D0403193D2942296E086F04031D93
:101280004229B829EC01ED01B00A0319B10AEE01B7
:10129000EF01803175268831003020003106031DB2
:1012A000532901303006031D7629B701B8012130DA
:1012B0002100DA000030DB00DC010F30DD000030FF
:1012C000DE0080313626883145302000A1005230C2
:1012D000A2004B30A3002030A4003230A5003030F3
:1012E000A6003130A7003830A800B82900303106F8
:1012F000031D7C2902303006031D83290130B7000D
:101300000030B800B82900303106031D89290330A8
:101310003006031DAA29B701B80121302100DA00E7
:101320000030DB00DC010F30DD000030DE008031FA
:101330003626883155302000A1004D30A2002030E3
:10134000A3004630A4004530A5005230A600493025
:10135000A700B82900303106031DB029043030063B
:10136000031DB8290130B7000030B800B001B10149
:1013700000306B06031DBE2932306A06031D782A31
:10138000370838040319D22900302100D0009830E2
:10139000D10022000D160C1110302100D6000030B3
:1013A000D700DF2921000030D0009030D10022008A
:1013B0000D120C1520302100D6000030D700D401CA
:1013C000D5012130DA000030DB008031562688312B
:1013D00071085502031DEE29700854020318782A7B
:1013E0002130540784000030553D85002030000234
:1013F000D200D3010030D33BBE01BF010130520700
:10140000F3000030533DF4007308F0007408F1005D
:10141000F035F10D1C307007F4008730713DF50098
:101420005208F0005308F100F035F10D1C30700740
:1014300084008730713D85000008F200013100080A
:10144000F30074088400750885000008F00001317D
:101450000008F10072087002F2007308713BF3009B
:1014600073083F02031D362A72083E020318742ACD
:10147000200066086704031D3E2A382A210052080E
:10148000F0005308F100F035F10D1C3070078400B6
:101490008730713D85000008F00001310008F1003F
:1014A0003E087007F3003F08713DF4007308F00038
:1014B0007408F100F035F10D7008500784007108D0
:1014C000513D85000008DA0001310008DB005608B4
:1014D000DC008031F92588312000E601E701210098
:1014E000BE0A0319BF0AFE29D40A0319D50AE12945
:0414F0002728792A06
:101594007D3084008A3085004530F0000130F10050
:1015A400213086000030870080310C278831DC3000
:1015B4008400873085001E30F0000130F100A03037
:1015C40086000030870080310C278831C2308400C7
:1015D4008A3085000830F0000130F1006630860062
:0C15E4000030870080310C27883108009F
:100E38000034003404340034073400340D340034F2
:100E4800173400341F3400342C3400343634003462
:100E5800393400343F340034453400344C340034E1
:100E680055340034593400345F340034623400346B
:100E78006834003470340034753400347D34003400
:100E8800853400348D340034953400349D34003476
:100E9800A5340034AD340034B5340034B8340034EB
:100EA800BC340034C5340034CE340034D734003474
:100EB800DF340034EE340034F934003403340134C0
:100EC8000F3401341A340134243401342E340134FB
:100ED8003A3401344534013448340134503401344F
:100EE8005B34013464340134713401347C340134AA
:100EF80088340134933401349F340134AA340134E2
:100F0800B4340134BF340134CA340134D534013423
:100F1800E6340134F2340134FD3401340634023449
:100F28000B34023411340234163402341D340234C2
:100F3800273402342B340234343402343C3402343F
:100F4800453402344D340234553402345B340234AF
:100F5800633402346B3402346E3402347234023433
:100F68007B3402347E3402348B34023493340234BA
:100F78009C340234A4340234AC340234B234023423
:100F8800BA340234BF340234C7340234D0340234A1
:100F9800DD340234E6340234EF340234F7340234F8
:100FA800FE34023401340334083403341134033476
:100FB8000034003400340034003400340034003489
:100FC8000034003400340034003400340034003479
:100FD8000034003400340034003400340034003469
:0C0FE800003400340034003400340034C5
:1014FA000034003400340034003400340034003442
:0E150A00003400340034003400340034003467
:041518000034003467
:0A151C0000340034003400340034C1
:041526000034003459
:0A152A0000340034003400340034B3
:0615340000340034003415
:10153A000034003400340034003400340034003401
:10154A0000340034003400340034003400340034F1
:10155A0000340034003400340034003400340034E1
:0C156A000034003400340034003400343D
:041576000034003409
:0A157A000034003400340034003463
:0415840000340034FB
:0415880000340034F7
:04158C0000340034F3
:0415900000340034EF
:102000000034003400340034003400340034003430
:10201000FE34D03400340034003400341E34003434
:1020200000340034003400341E34003400340034F2
:1020300000340034003480341034F034F034803410
:102040001E3480341034F034F03480341E34803444
:102050001034003400340034003400343C34603434
:1020600042341034C234F8347F34103442341034E3
:102070008C34E03400340034003400343C34003418
:10208000423400344234103442346034BC3480343E
:1020900040340034B034E0344C3410344234103422
:1020A000403410348034E0340034003400340034E0
:1020B0008034E0345C341034223410346234103410
:1020C000A23410341C34A034003460348034903492
:1020D00000340034003400341E3400340034003442
:1020E00000340034E034E034183418340434043458
:1020F0000234023400340034003400340234023438
:102100000434043418341834E034E0340034003437
:102110000034003404340034383400340E340034D5
:1021200038340034043400340034003400340034D3
:10213000403400344034003440340034F834C03487
:10214000403400344034003440340034003400342F
:10215000003400340034023400341C3400340034C1
:10216000003400348034003480340034803400344F
:10217000803400340034003400340034003410342F
:10218000003400340034003400347034C0348034FF
:102190003834003406340034003400340034003461
:1021A000FC34E0340234103402341034023410347D
:1021B00002341034FC34E034003400340034003491
:1021C0000434003404340034FE34F0340034003479
:1021D000003400340C34303402345034023490343F
:1021E00082341034423410343C341034003400341F
:1021F000003400340C34603402341034423410346F
:102200004234103442341034BC34E03400340034EE
:1022100000340034803480346034803410348034AE
:102220000C348034FE34F034003480340034003414
:10223000003400347E3460342234103422341034BC
:102240002234103422341034C234E03400340034E8
:1022500000340034FC34E03442341034223410347E
:102260002234103422341034CC34E03400340034BE
:102270000034003402340034023410340234E034C8
:10228000C2340034323400340E34003400340034AC
:1022900000340034BC34E03442341034423410345E
:1022A0004234103442341034BC34E034003400344E
:1022B000003400347C34603482341034823410347E
:1022C0008234103442341034FC34E03400340034AE
:1022D000003400341034103400340034003400343E
:1022E0000034023410341C34003400340034003420
:1022F00040340034A0340034A0340034103480342E
:10230000103480340834403408344034003400340D
:10231000003400349034003490340034903400346D
:1023200090340034903400349034003490340034CD
:10233000003400340034003408344034083440346D
:102340001034803410348034A0340034A03400348D
:102350004034003400340034003400340C34003491
:102360000234003402340034C23490342234003455
:102370001C3400340034003400340034C034E03401
:1023800030341834083404348434E434643412347B
:102390001234123412341234123422341234F2341D
:1023A000F43412340434143418342034E034C03497
:1023B0000034003400340034003430340034C0348D
:1023C000E0340034983400348634003498340034D7
:1023D000E03400340034C03400343034003400348D
:1023E00000340034FE34F0344234103442341034BB
:1023F000423410344234103442341034A434203483
:102400001834C0340034003400340034F0348034E4
:102410000C34603404342034023410340234103468
:102420000234103402341034043420340C34603458
:10243000103480340034003400340034FE34F0347E
:1024400002341034023410340234103402341034A4
:1024500002341034043420340C346034F0348034CA
:102460000034003400340034FE34F034423410348C
:102470004234103442341034423410344234103474
:102480004234103402341034003400340034003448
:10249000FE34F034423400344234003442340034E8
:1024A00042340034423400344234003402340034C4
:1024B0000034003400340034F03480340C346034A0
:1024C0000434203402341034023410340234103412
:1024D000423410344234103444342034C834F0349C
:1024E0000034003400340034FE34F034403400341E
:1024F000403400344034003440340034403400343C
:102500004034003440340034FE34F03400340034BD
:1025100000340034FE34F03400340034003400342D
:10252000003460340034103400341034003410347B
:1025300000341034FE34E03400340034003400340D
:10254000FE34F034803400344034003460340034DD
:10255000903400340834803404344034023420345D
:10256000003410340034003400340034FE34F034CD
:10257000003410340034103400341034003410347B
:10258000003410340034103400340034003400348B
:10259000FE34F0340834003430340034C0340034B5
:1025A0000034C034003430340034C034C03400341B
:1025B0003034003408340034FE34F0340034003455
:1025C00000340034FE34F034043400340834003471
:1025D00030340034403400348034803400344034AB
:1025E00000342034FE34F03400340034003400343D
:1025F000F03480340C346034043420340234103429
:1026000002341034023410340234103404342034D0
:102610000C346034F034803400340034003400343E
:10262000FE34F03482340034823400348234003496
:102630008234003482340034823400344434003430
:10264000383400340034003400340034F034803442
:102650000C34603404342034023410340234103426
:102660000234903402345034043420340C34703446
:10267000F03488340034003400340034FE34F03454
:1026800042340034423400344234003442340034A2
:1026900042340034E43400341834E034003410346C
:1026A00000340034003400341834403424342034EE
:1026B0004234103442341034423410344234103432
:1026C000843420340834C0340034003400340034FE
:1026D0000234003402340034023400340234003452
:1026E000FE34F03402340034023400340234003456
:1026F000023400340034003400340034FE34C0347A
:1027000000342034003410340034103400341034D9
:10271000003410340034103400342034FE34C0341B
:1027200000340034003400340634003418340034EB
:10273000E03400340034C034003430340034C03469
:10274000E0340034183400340634003400340034EB
:10275000003400340E34003470340034803480345B
:1027600000347034803480346034003418340034E1
:10277000063400341834003460340034803480343B
:102780000034703480348034703400340E340034BB
:102790000034003400340034023410340434203463
:1027A0000834403410348034E0340034E0340034F1
:1027B000103480340834403404342034023410346B
:1027C000003400340034003406340034083400345B
:1027D0001034003420340034C034F0342034003459
:1027E000103400340834003406340034003400342B
:1027F00000340034023430340234503482349034A3
:1028000042341034323410340A3410340634103464
:102810000034003400340034FE34FE340234023418
:1028200002340234003400340034003406340034FE
:1028300038340034C0348034003470340034003410
:10284000003400340234023402340234FE34FE34E4
:1028500000340034003400340834003404340034CC
:1028600002340034043400340834003400340034BA
:1028700000340034003402340034023400340234B2
:1028800000340234003402340034023400340234A0
:102890000034023400340034003400340234003494
:1028A0000434003400340034003400342034E03484
:1028B00090341034903410349034103490341034F8
:1028C000E034E03400341034003400340034003498
:1028D000FE34F034203420341034103410341034EA
:1028E00010341034E034E034003400340034003468
:1028F000C034C03420342034103410341034103438
:102900001034103420342034403440340034003447
:1029100000340034E034E034103410341034103417
:102920001034103420342034FE34F03400340034B9
:1029300000340034C034C034A03420349034103417
:1029400090341034A0342034C03440340034003487
:102950000034003410340034FC34F03412340034C9
:10296000023400340034003400340034E034E03405
:10297000103412341034123410341234203422340F
:10298000F034FC340034003400340034FE34F034CD
:102990002034003410340034103400341034003447
:1029A000E034F0340034003400340034F234F034D5
:1029B000003400340034003400340234F234FC3487
:1029C0000034003400340034FE34F03400348034F9
:1029D0008034003440348034203440341034203487
:1029E000003410340034003400340034FE34F03449
:1029F0000034003400340034F034F0342034003437
:102A0000103400341034003410340034E034F03426
:102A100020340034103400341034003410340034C6
:102A2000E034F0340034003400340034F034F03456
:102A300020340034103400341034003410340034A6
:102A4000E034F0340034003400340034C034C03496
:102A50002034203410341034103410341034103436
:102A600020342034C034C034003400340034003406
:102A7000F034FE3420342034103410341034103448
:102A800010341034E034E0340034003400340034C6
:102A9000E034E03410341034103410341034103476
:102AA00020342034F034FE34003400340034003458
:102AB000F034F03420340034103400341034003456
:102AC0000034003400340034603420349034103446
:102AD00090341034103490341034903420346034F6
:102AE000003400340034003410340034FC34E0345A
:102AF000103410340034003400340034F034E03446
:102B000000341034003410340034103400342034D5
:102B1000F034F03400340034003400343034003405
:102B2000C03400340034C034003430340034C03495
:102B3000C034003430340034003400340034003405
:102B400030340034C03480340034703400344034C5
:102B5000C034803430340034C034803400344034E5
:102B600000347034C03480343034003400340034E5
:102B700000340034103410342034203440344034D5
:102B800080348034403440342034203410341034C5
:102B9000003400340034003430340234C0340234A1
:102BA0000034C434003438340034C034C034003409
:102BB0003034003400340034003400341034303405
:102BC0001034503410349034903410345034103465
:102BD0003034103400340034003400348034003495
:102BE000803400347C34FC34023402340234023445
:102BF0000034003400340034FE34FE340034003439
:102C00000034003402340234023402347C34FC34A4
:102C10008034003480340034003400340034003414
:102C20000C340034023400340234003404340034F0
:102C300008340034083400340634003400340034DE
:042C40000034003428
:103000000034003400340034003400340034003420
:103010000B347F340034003400340034003478340E
:103020000034003400340034003478340034003488
:1030300000340034013400340F34083401340F34C8
:10304000013478340F34083401340F3401347834C7
:1030500000340834003400340034003406343C3486
:10306000083442341F3443340834FE3408344234C4
:1030700007343134003400340034003400343C343C
:1030800000344234083442340634423401343D348E
:103090000034023407340D340834323408344234F6
:1030A000083402340734013400340034003400346E
:1030B0000734013408343A3408344434083446348C
:1030C00008344534053438340634003409340134C6
:1030D00000340034003400340034783400340034D8
:1030E00000340034073407341834183420342034C2
:1030F0004034403400340034003400344034403430
:1031000020342034183418340734073400340034A1
:10311000003400340034203400341C340034703463
:1031200000341C34003420340034003400340034C3
:1031300000340234003402340034023403341F34C7
:1031400000340234003402340034023400340034D9
:103150000034003440340034383400340034003457
:1031600000340034003401340034013400340134BC
:1031700000340134003400340034003408340034A6
:1031800000340034003400340E340034013403348D
:1031900000341C3400346034003400340034003413
:1031A00007343F3408344034083440340834403461
:1031B0000834403407343F340034003400340034E1
:1031C00000342034003420340F347F340034003491
:1031D000003400340C3430340A3440340934403480
:1031E000083441340834423408343C340034003468
:1031F0000034003406343034083440340834423467
:10320000083442340834423407343D340034003446
:1032100000340034013401340134063401340834FC
:10322000013430340F347F3401340034003400343E
:103230000034003406347E340834443408344434D2
:1032400008344434083444340734433400340034FC
:103250000034003407343F340834423408344434F2
:1032600008344434083444340734333400340034EC
:1032700000340034003440340834403407344034DF
:103280000034433400344C3400347034003400349F
:103290000034003407343D340834423408344234B6
:1032A000083442340834423407343D3400340034A6
:1032B0000034003406343E34083441340834413498
:1032C000083441340834423407343F340034003485
:1032D000003400340834083400340034003400343E
:1032E00040340034383408340034003400340034BE
:1032F0000034023400340534003405340134083419
:1033000001340834023410340234103400340034F0
:1033100000340034003409340034093400340934F2
:1033200000340934003409340034093400340934D9
:1033300000340034003400340234103402341034C9
:1033400001340834013408340034053400340534C1
:10335000003402340034003400340034003430349B
:1033600000344034003440340934433400344434AD
:10337000003438340034003400340034073403346B
:1033800018340C3420341034273421344834263493
:103390004834483448344834443448344F3448344A
:1033A00048342F3428342034043418340334073498
:1033B00000340034003400340C340034033400345E
:1033C00000340734003419340034613400341934C3
:1033D00000340734033400340C3400340034003437
:1033E000003400340F347F3408344234083442341B
:1033F0000834423408344234083442340434253426
:1034000003341834003400340034003401340F34F1
:103410000634303404342034083440340834403422
:103420000834403408344034043420340634303412
:103430000134083400340034003400340F347F3455
:1034400008344034083440340834403408344034BC
:1034500008344034043420340634303401340F341A
:1034600000340034003400340F347F3408344234E4
:103470000834423408344234083442340834423484
:10348000083442340834403400340034003400340A
:103490000F347F3400344234003442340034423438
:1034A0000034423400344234003442340034403476
:1034B000003400340034003401340F340634303426
:1034C0000434203408344034083440340834403460
:1034D0000834423408344234043422340F34133470
:1034E00000340034003400340F347F3400340234AC
:1034F0000034023400340234003402340034023424
:1035000000340234003402340F347F340034003489
:10351000003400340F347F3400340034003400347D
:1035200006340034083400340834003408340034DD
:103530000834003407347F3400340034003400345D
:103540000F347F3400340134003402340034063444
:10355000003409340134103402342034043440344B
:103560000834003400340034003400340F347F3425
:10357000083400340834003408340034083400348B
:10358000083400340834003400340034003400348B
:103590000F347F340034103400340C3400340334DE
:1035A000033400340C340034033400340034033466
:1035B00000340C34003410340F347F3400340034C1
:1035C000003400340F347F3400342034003410349D
:1035D00000340C3400340234013401340234003439
:1035E000043400340F347F340034003400340034A9
:1035F00001340F3406343034043420340834403479
:10360000083440340834403408344034043420341E
:103610000634303401340F340034003400340034C4
:103620000F347F34003441340034413400344134A9
:103630000034413400344134003441340034223405
:1036400000341C34003400340034003401340F34AE
:1036500006343034043420340834403408344034E0
:10366000093440340A344034043420340E343034C5
:1036700011340F3400340034003400340F347F34FC
:103680000034423400344234003442340034423492
:1036900000344234003427340734183408340034FA
:1036A0000034003400340034023418340434243438
:1036B0000834423408344234083442340834423442
:1036C0000434213403341034003400340034003422
:1036D000003440340034403400344034003440344A
:1036E0000F347F34003440340034403400344034EC
:1036F00000344034003400340034003403347F3468
:1037000004340034083400340834003408340034FD
:1037100008340034083400340434003403347F3473
:103720000034003400340034003460340034183481
:1037300000340734033400340C34003403340034D0
:10374000003407340034183400346034003400345A
:10375000003400340034703400340E340134013449
:103760000E3400340134013400340634003418348B
:103770000034603400341834003406340134013429
:103780000E3400340134013400340E34003470340B
:10379000003400340034003408344034043420341D
:1037A0000234103401340834003407340034073450
:1037B00001340834023410340434203408344034E2
:1037C00000340034003400340034603400341034E9
:1037D00000340834003404340F3403340034043427
:1037E00000340834003410340034603400340034C1
:1037F000003400340C3440340A3440340934413449
:103800000834423408344C340834503408346034BA
:1038100000340034003400347F347F34403440348A
:103820004034403400340034003400340034603418
:1038300000341C34013403340E34003400340034BA
:103840000034003440344034403440347F347F34DA
:103850000034003400340034003410340034203498
:103860000034403400342034003410340034003448
:1038700000340034403400344034003440340034E8
:103880004034003440340034403400344034003498
:103890004034003400340034003400340034403408
:1038A000003420340034003400340034073404344D
:1038B0000834093408340934083409340834093424
:1038C0000734073408340034003400340034003442
:1038D0000F347F3404340434083408340834083492
:1038E000083408340734073400340034003400341A
:1038F00003340334043404340834083408340834FA
:1039000008340834043404340234023400340034FB
:1039100000340034073407340834083408340834D9
:1039200008340834043404340F347F340034003451
:1039300000340034033403340434053408340934C7
:1039400008340934043405340234033400340034B8
:1039500000340034003408340F343F340034483429
:103960000034403400340034003400340734073469
:10397000483408344834083448340834443404346F
:103980003F340F3400340034003400340F347F34BB
:10399000003404340034083400340834003408346B
:1039A0000F34073400340034003400340F344F3403
:1039B0000034003400340034403400343F344F3499
:1039C00000340034003400340F347F3401340034C8
:1039D0000034013401340234023404340434083431
:1039E0000834003400340034003400340F347F34A1
:1039F00000340034003400340F340F340034043405
:103A00000034083400340834003408340F340734E8
:103A100000340434003408340034083400340834EA
:103A20000F34073400340034003400340F340F34C2
:103A300000340434003408340034083400340834CA
:103A40000F340734003400340034003403340334BA
:103A5000043404340834083408340834083408348E
:103A600004340434033403340034003400340034A8
:103A70007F340F34043404340834083408340834F0
:103A80000834083407340734003400340034003478
:103A90000734073408340834083408340834083448
:103AA000043404347F340F340034003400340034E0
:103AB0000F340F3400340434003408340034083434
:103AC000003400340034003404340634083409343B
:103AD0000834093409340834093408340634043409
:103AE00000340034003400340034083407343F34E8
:103AF00008340834003400340034003407340F3400
:103B000008340034083400340834003404340034F9
:103B10000F340F34003400340034003400340C34DB
:103B200000340334033400340C34003403340034E0
:103B30000034033400340C340034003400340034D6
:103B400000340C34013403340E34003402340034B5
:103B50000134033400340C340134033402340034AF
:103B60000E3400340134033400340C340034003497
:103B70000034003408340834043404340234023489
:103B80000134013402340234043404340834083477
:103B9000003400340034003440340C3440340334F6
:103BA000233400341C340034033400340034033430
:103BB00000340C3400340034003400340C34083445
:103BC0000A340834093408340834093408340A340F
:103BD00008340C3400340034003400340034013430
:103BE000003401343F343E344034403440344034B7
:103BF00000340034003400347F347F340034003427
:103C00000034003440344034403440343F343E3497
:103C10000034013400340134003400340034003402
:103C20000034303400344034003440340034203424
:103C30000034103400341034003460340034003464
:043C40000034003418
:020000040001F9
:06000E00A408871D1F3F3E
:00000001FF
